:100000000C9460010C9488010C9488010C94880174
:100010000C9488010C9488010C9488010C9488013C
:100020000C9488010C9488010C947D060C9449056D
:100030000C9488010C9488010C9488010C9488011C
:100040000C9488010C9488010C9488010C9488010C
:100050000C9488010C9488010C9488010C94A201E2
:100060000C9488010C9488010C9488010C948801EC
:100070000C9488010C9488010C9488010C948801DC
:100080000C9488010C9488010C9488010C948801CC
:100090000C9488010C9488010C9488010C948801BC
:1000A0000C9488010C9488010C948801A502A80284
:1000B00097029B02A102C902C902C902AC02B002A6
:1000C000B402BA02BE02C902C40200000002000962
:1000D0000F0000030401000C00000408020110409E
:1000E00080401020408040800802040180402010A1
:1000F000020110801020404004040404040304059D
:1001000002020202040302020202060606060606B4
:1001100004040202020400000000250028002B0055
:100120002E00310000000000240027002A002D00CE
:10013000300000C18081C112010002020000404F66
:100140001B069200010102000112010002000000E2
:10015000404F1B0692000101020001537061726B57
:1001600046756E00537061726B46756E2050726FEB
:10017000204D6963726F0004030904080B0002023A
:100180000201000904000001020200000524001021
:1001900001052401010104240206052406000107CB
:1001A00005810310004009040100020A0000000755
:1001B0000502024000000705830240000000000025
:1001C00000000000002A2B280000000000000000B2
:1001D000000000000000000000000000002C9EB4A1
:1001E000A0A1A2A434A6A7A5AE362D3738271E1F7E
:1001F00020212223242526B333B62EB7B89F848529
:10020000868788898A8B8C8D8E8F90919293949516
:10021000969798999A9B9C9D2F3130A3AD350405F4
:10022000060708090A0B0C0D0E0F101112131415F6
:10023000161718191A1B1C1DAFB1B0B5000904021E
:1002400000010300000009210101000122650007EF
:1002500005840340000105010902A1010901A10073
:10026000850105091901290315002501950375016B
:1002700081029501750581030501093009310938AD
:100280001581257F750895038106C0C00501090603
:10029000A1018502050719E029E71500250175016F
:1002A000950881029501750881039506750815006A
:1002B00025650507190029658100C000AF070209FF
:1002C00011241FBECFEFDAE0DEBFCDBF11E0A0E00A
:1002D000B1E0EEE7F2E102C005900D92A832B1075D
:1002E000D9F721E0A8E2B1E001C01D92A739B20719
:1002F000E1F712E0C0ECD2E004C02297FE010E94B8
:100300003909CC3BD107C9F70E943A030C943D0947
:100310000C94000061E083E00C94CA0261E083E089
:100320000E94030368EE73E080E090E00E940F02F9
:1003300060E083E00E94030368EE73E080E090E0F9
:100340000C940F021F920F920FB60F9211242F934D
:100350003F938F939F93AF93BF9380912901909187
:100360002A01A0912B01B0912C013091280123E0AA
:10037000230F2D3720F40196A11DB11D05C026E8DD
:10038000230F0296A11DB11D2093280180932901FE
:1003900090932A01A0932B01B0932C0180912D0101
:1003A00090912E01A0912F01B09130010196A11DD5
:1003B000B11D80932D0190932E01A0932F01B09336
:1003C0003001BF91AF919F918F913F912F910F90ED
:1003D0000FBE0F901F9018953FB7F89480912D0194
:1003E00090912E01A0912F01B091300126B5A89BCC
:1003F00005C02F3F19F00196A11DB11D3FBF662713
:10040000782F892F9A2F620F711D811D911D42E057
:10041000660F771F881F991F4A95D1F70895CF92CD
:10042000DF92EF92FF92CF93DF936B017C010E94EA
:10043000EC01EB01C114D104E104F10489F00E9444
:10044000F1060E94EC016C1B7D0B683E734090F33B
:1004500081E0C81AD108E108F108C851DC4FEACFA1
:10046000DF91CF91FF90EF90DF90CF900895789437
:1004700084B5826084BD84B5816084BD85B58260A9
:1004800085BD85B5816085BDEEE6F0E08081816047
:100490008083E1E8F0E01082808182608083808147
:1004A00081608083E0E8F0E0808181608083E1E921
:1004B000F0E0808182608083808181608083E0E9D8
:1004C000F0E0808181608083E1ECF0E080818460F5
:1004D0008083808182608083808181608083E3EC7F
:1004E000F0E0808181608083E0ECF0E080818260D8
:1004F0008083E2ECF0E0808181608083EAE7F0E0D5
:10050000808184608083808182608083808181603B
:100510008083808180688083089590E0FC0131971A
:10052000EF30F105B0F5EA5AFF4F0C94370980918E
:1005300080008F7703C0809180008F7D8093800042
:10054000089580918000877FF9CF84B58F7702C0AE
:1005500084B58F7D84BD0895809190008F7707C00A
:10056000809190008F7D03C080919000877F809361
:10057000900008958091C0008F7703C08091C000E3
:100580008F7D8093C00008958091C200877F809303
:10059000C2000895CF93DF9390E0FC01E652FF4F35
:1005A0002491FC01E850FF4F8491882349F190E0A9
:1005B000880F991FFC01EC5DFE4FA591B4918A5EF6
:1005C0009E4FFC01C591D4919FB7611108C0F8946A
:1005D0008C91209582238C93888182230AC062307B
:1005E00051F4F8948C91322F309583238C93888129
:1005F000822B888304C0F8948C91822B8C939FBFAC
:10060000DF91CF9108950F931F93CF93DF931F92A4
:10061000CDB7DEB7282F30E0F901E653FF4F8491C4
:10062000F901E652FF4F1491F901E850FF4F049190
:100630000023C9F0882321F069830E948D0269811B
:10064000E02FF0E0EE0FFF1FEA5EFE4FA591B491A0
:100650009FB7F8948C91611103C01095812301C05C
:10066000812B8C939FBF0F90DF91CF911F910F91A2
:10067000089508950E9437020E94390381E391E0B2
:100680000E94D3060E948A01C0E0D0E00E948E0141
:100690002097E1F30E940000F9CF4091350150917D
:1006A0003601209133013091340142175307B4F4DD
:1006B0009091E8009570E1F39091E80092FD19C0E7
:1006C0008093F100809135019091360101968F73EE
:1006D0009927892B19F48EEF8093E80080913501DA
:1006E000909136010196909336018093350181E017
:1006F000089580E00895CF92DF92FF920F931F93A9
:10070000CF93DF931F92CDB7DEB7082F162F862F1A
:10071000880F8E5F99830E944D0383E00E944D03F2
:10072000F02EC02E9981D92E8C2D8F19811778F437
:10073000F60184910E944D03082F80E00E944D0332
:100740008023FFEFCF1ADF0A8111EECF01C081E0D5
:100750000F90DF91CF911F910F91FF90DF90CF907D
:100760000895615030F02091F100FC012083019642
:10077000F8CF289884E68093380108952FB7FC01BC
:100780002083F89467706093E9000895CF93DF9316
:100790001F92CDB7DEB7682FCE0101960E94BE032F
:1007A0008091F20099819FBF0F90DF91CF910895C2
:1007B000FF920F931F93CF93DF9300D0CDB7DEB797
:1007C000F62E8A0190913701992311F057FF03C04B
:1007D0008FEF9FEF2BC0682FCE0101967A830E9486
:1007E000BE038091F20090E0A8017A818017910702
:1007F0000CF4AC01EF2DF72FF40E84E6FE1639F061
:100800002898809338019091F1009193F7CF41158A
:10081000510521F08091F200882321F089818FBF5A
:10082000CA0104C08BE68093E800F8CF0F900F90C8
:10083000DF91CF911F910F91FF900895CF93DF9398
:100840001F92CDB7DEB741E050E0BE016F5F7F4F32
:100850000E94D803019719F4898190E002C08FEFBC
:100860009FEF0F90DF91CF910895CF93DF931F9269
:10087000CDB7DEB7682FCE0101960E94BE039091DE
:10088000E800892F807295FF04C09091F20080E407
:10089000891B99819FBF0F90DF91CF9108956F922F
:1008A0007F928F929F92AF92BF92CF92DF92EF9200
:1008B000FF920F931F93CF93DF931F92CDB7DEB7B5
:1008C000782E7B01C42EB52E80913701882369F0E4
:1008D000042F152F8AEFD82E872D8072982E9AE339
:1008E000A92E872D8074882E11C08FEF9FEF57C0DF
:1008F000872D0E943504682E81110CC0DA94A9F36B
:1009000061E070E080E090E00E940F0201151105A7
:1009100079F73BC0282F30E0021713070CF4602E44
:10092000672DCE0101960E94BE038091E80085FFED
:1009300029C0262D30E0021B130B992039F06A9450
:100940008FEF6816B1F01092F100F9CFF701862D04
:1009500077FE07C0815058F094919093F100319642
:10096000F9CF815020F091919093F100FACFE20EEF
:10097000F31E8091E80085FF0FC00115110511F4E9
:1009800081100AC089818FBFC1CF5D9884E68093B2
:1009900039018C2D9B2D03C0A092E800F3CF0F905E
:1009A000DF91CF911F910F91FF90EF90DF90CF904B
:1009B000BF90AF909F908F907F906F90089510920E
:1009C000E900109236011092350190933401809322
:1009D00033010895CF92DF92FF920F931F93CF932D
:1009E000DF9300D0CDB7DEB7F82E8A016B01011579
:1009F0001105B1F0F601F7FE02C0849101C08081BB
:100A000049835A830E944D0301501109FFEFCF1A09
:100A1000DF0A49815A818111EACF8FEF9FEF01C030
:100A2000CA010F900F90DF91CF911F910F91FF900E
:100A3000DF90CF9008951F93CF93DF931F92CDB790
:100A4000DEB7162F2091E80022FFFCCF612F7983BB
:100A50000E94B1038BEF8093E800812F7981972F5B
:100A60000F90DF91CF911F910895CF93DF931F9245
:100A7000CDB7DEB71982CE0101960E944F07CE0195
:100A800001960E94EA07898190E00F90DF91CF9153
:100A900008951F920F920FB60F921124EF92FF92BA
:100AA0000F931F932F933F934F935F936F937F9376
:100AB0008F939F93AF93BF93EF93FF93CF93DF9366
:100AC000CDB7DEB76297DEBFCDBF1092E90080914F
:100AD000E80083FFEBC068E0CE010A960E94B103F4
:100AE00082EF8093E8009A8597FF05C08091E80027
:100AF00080FFFCCF03C08EEF8093E800892F8076C3
:100B000009F0B9C08B85811105C01092F1001092D7
:100B1000F100C5C0282F2D7F213009F4C0C08530D9
:100B200049F48091E80080FFFCCF8C858068809339
:100B3000E300B5C0863009F076C02D85E888F988D5
:100B4000223071F580E090E02A8B0E94DF040E9441
:100B5000350599E08E010F5F1F4FF801392F119273
:100B60003A95E9F799832A892A8391E09E8390E850
:100B700098879AEF99872091350130913601275F48
:100B80003F4F3C832B838D83C7010E94DF0449E0E4
:100B900050E0B80180E00E94EA040E9435057FC061
:100BA000C7012A8B0E94DF042A89223241F482E2A3
:100BB00090E00E94F507892B09F071C074C02130C4
:100BC00069F488899989089711F4209332018091FA
:100BD0003201811118C069E471E01AC0233009F0B4
:100BE00062C08C85882391F0823021F462E184E632
:100BF00091E006C0813009F056C068E08BE591E0D5
:100C00000E947B034AC067E371E002C067E771E0BE
:100C10006115710509F447C0FB01449150E080E87B
:100C20000E94EA043CC0873009F43DC0883021F4BA
:100C300081E08093F10033C0893089F5937099F594
:100C4000E3E3F1E081E021E096E38093E900209383
:100C5000EB0034913093EC009093ED008F5F319670
:100C6000853099F78EE78093EA001092EA008C8530
:100C70008093370114C0888999890E94DF048E858A
:100C8000811105C0CE010A960E945A0706C0823023
:100C900051F4CE010A960E941D08882321F08EEFA0
:100CA0008093E80003C081E28093EB0062960FB668
:100CB000F894DEBF0FBECDBFDF91CF91FF91EF91D2
:100CC000BF91AF919F918F917F916F915F914F9164
:100CD0003F912F911F910F91FF90EF900F900FBEBA
:100CE0000F901F9018958093E9008091F20088235F
:100CF00019F08AE38093E80008951F920F920FB6CF
:100D00000F9211242F933F934F935F936F937F9391
:100D10008F939F93AF93BF93EF93FF938091E100E5
:100D20001092E10083FF0FC01092E90091E09093D0
:100D3000EB001092EC0092E39093ED0010923701DB
:100D400098E09093F00082FF1DC083E00E9473063C
:100D500080913901882339F0809139018150809345
:100D60003901882369F080913801882359F08091F6
:100D70003801815080933801811104C0289A02C043
:100D80005D9AF1CFFF91EF91BF91AF919F918F91BC
:100D90007F916F915F914F913F912F910F900FBE77
:100DA0000F901F9018951092370181E08093D70023
:100DB00080EA8093D80082E189BD09B400FEFDCFAE
:100DC00061E070E080E090E00E940F0280E9809393
:100DD000D8008CE08093E2001092E000559A209AAF
:100DE00008950895CF93DF931F92CDB7DEB769833F
:100DF000DC01ED91FC910280F381E02D41E050E0B7
:100E0000BE016F5F7F4F09950F90DF91CF910895DD
:100E1000CF93DF93EC018C859D8597FF05C082E021
:100E20000E941E049D878C878C859D85DF91CF91C4
:100E3000089583E00C947306FC018485958597FDE5
:100E400006C082E00E94C60390E00196089582E009
:100E50000E94C60390E00895FC018485958597FD66
:100E600005C02FEF3FEF35872487089582E00C946B
:100E70001E04CF93DF93EC0180910701882331F0AA
:100E800083E00E944F041816190634F081E090E0C8
:100E90009B838A8380E090E0DF91CF910895FC01ED
:100EA00020812E5F208342E450E06BE771E080E810
:100EB0000C94EA04FC0181819081913A59F48132C9
:100EC00009F03CC047E050E060E071E080E00E9443
:100ED000EA0443C0913291F5803239F467E070E062
:100EE00080E091E00E941B0506C0823209F035C007
:100EF0008281809307018091000190910101A0916E
:100F00000201B0910301803B9440A105B105C1F4F9
:100F10008091070180FD14C087E797E7909301084F
:100F2000809300082BE088E190E00FB6F894A89534
:100F3000809360000FBE209360000FC080E0089592
:100F400088E10FB6F89480936000109260000FBEA5
:100F5000A895109201081092000881E0089510925F
:100F60003D0110923C0188EE93E0A0E0B0E0809358
:100F70003E0190933F01A0934001B09341018EE068
:100F800091E090933B0180933A018FEF9FEF909314
:100F90004701809346010895FF920F931F93CF93CB
:100FA000DF93EC01F62EE881F9810480F581E02DD4
:100FB00009958C01E881F9810680F781E02D6F2D7C
:100FC000CE010995C8019927DF91CF911F910F910B
:100FD000FF900895FC0120812F5F208349E150E0BC
:100FE0006DE372E080E80C94EA0445E650E066E5C3
:100FF00072E080E80C94EA04EF92FF920F931F9343
:10100000CF93DF931F92CDB7DEB789838B017A012F
:1010100041E050E0BE016F5F7F4F84E00E944F04CB
:10102000A701B80184E40E944F040F90DF91CF9193
:101030001F910F91FF90EF900895FC0191818081A5
:10104000813A31F481E0913091F0933089F411C00C
:10105000813271F49B3021F482818093090105C0B3
:101060009A3031F482818093080181E008950895D7
:1010700080E0089548E050E082E00C94FC07CF93B4
:10108000DF93DC01683818F0E8E7E60F25C0E62FAB
:10109000F0E067FF11C0E058F10981E090E001C085
:1010A000880FEA95EAF714969C911497982B14965A
:1010B0009C931497E0E010C0E354FE4FE491EE23BC
:1010C00009F440C0E7FF08C014968C911497826021
:1010D00014968C931497EF7716968C9116978E171B
:1010E00041F117968C9117978E1719F118968C91DC
:1010F00018978E17F1F019968C9119978E17C9F0E1
:101100001A968C911A978E17A1F01B968C911B97AB
:101110008E1779F080E090E0ED01C80FD91F2E8185
:10112000211102C0EE8305C0019686309105A1F71A
:1011300009C0BD016C5F7F4FCD010E943A0881E07C
:1011400090E008C081E090E013969C938E931297F4
:1011500080E090E0DF91CF910895683818F0E8E7DB
:10116000E60F25C0E62FF0E067FF12C0E058F10956
:1011700021E030E001C0220FEA95EAF72095DC017A
:1011800014963C911497322314963C93E0E00FC0E0
:10119000E354FE4FE491EE2329F1E7FF08C0DC01A0
:1011A00014962C9114972D7F14962C93EF7720E0B2
:1011B00030E0EE2351F0DC01A20FB31F16964C91E4
:1011C00016974E1302C016961C922F5F3F4F263083
:1011D000310579F7BC016C5F7F4F0E943A0881E0CE
:1011E00090E0089580E090E00895FC011682178257
:1011F00010861186128613861482BC016C5F7F4FA5
:101200000C943A081092960110928D0110928C0164
:101210008EE191E090938B0180938A010895CF92A3
:10122000DF92EF92FF920F931F93CF93DF936C01A6
:101230007A01EB01E60EF71E00E010E0CE15DF05A7
:1012400061F06991D601ED91FC910190F081E02D62
:10125000C6010995080F191FF1CFC801DF91CF9181
:101260001F910F91FF90EF90DF90CF900895EE0FB8
:0E127000FF1F0590F491E02D0994F894FFCF34
:10127E0000E1000000000000010100000000F20685
:10128E0039071C072C070807190700000000CC07B8
:08129E000F093F08AD08F50837
:00000001FF
